:020000040000FA
:0400000013EF00F00A
:08000800006ED8CF02F0E0CF3A
:1000100001F0F2B281EC00F000D001C0E0FF00502E
:1000200002C0D8FF1000806A816A826A0F0EC16E1A
:100030000F6A39D85DD8D09EF28EF28C00000FB0D6
:1000400002D80000FBD70F90080E036E81948298AF
:10005000829482908090050E046E11EE00F020EEE6
:1000600010F0E6CFDEFF042EFCD7829E8198829AA4
:1000700082968292809210BE818811BE828A12BEC0
:10008000828613BE828214BE8082828E1046114602
:10009000124613461446032EE8D781848288828450
:1000A00082808080120093968186949E829E949C8A
:1000B0009398949A949694929292939494989494F8
:1000C000949092908198829A829682928092818472
:1000D0008288828482808080050E046E01EE00F0AA
:1000E000000EEE6E042EFCD7829C828C819612004C
:1000F00093809382F18CF292F288066A080E076E62
:10010000120086EC00F0F292F2881200D89081B2D0
:10011000D8800B320650056ED8900536010ED8B047
:10012000E828FA6E2E0E0524D8B0FA2AF96E02D00D
:100130000AD016D0072E1200010E066E060E076EAC
:100140000B50086E1200072E1200020E066E080EEB
:10015000076E0B50096ED8900932D8900932120000
:10016000072E1200000E066E080E076E100E0862B3
:1001700012000B500A6E01EE00F009500AC0EBFFAE
:100180000F8012000A0E0C6E010E0E6EC80E0D6E60
:10019000000000000D2EFCD70E2EF8D70C2EF4D741
:1001A00012000A0E0C6EFA0E0E6EC80E0D6E0000D6
:1001B00000000D2EFCD70E2EF8D70C2EF4D712000F
:1001C0000A0E0C6E0E6EC80E0D6E000000000D2E95
:1001D000FCD70E2EF8D70C2EF5D712000A0E0C6E97
:1001E000010E0E6E320E0D6E000000000D2EFCD7BB
:1001F0000E2EF8D70C2EF4D71200D1EC00F0D1EC73
:0C02000000F0D1EC00F0D1EC00F0120096
:020000040030CA
:0E000000FFFEFEFAFFFEFBFFFFFFFFFFFFFF0C
:00000001FF
